:100000000C94A2010C94E9010C94E9010C94E9010F
:100010000C94E9010C94E9010C94E9010C94E901B8
:100020000C94E9010C94E9010C94CF210C94A322C7
:100030000C943C1A0C94E9010C94E9010C94E9012C
:100040000C94E9010C94E9010C94E9010C94E90188
:100050000C94E9010C94871A0C94E9010C94E901C1
:100060000C94E9010C94E9010C94E9010C94E90168
:100070000C94E9010C94E9010C94E9010C94E90158
:100080000C94E9010C94E9010C94E9010C94E90148
:100090000C94E9010C94E9010C94E9010C94E90138
:1000A0000C94E9010C94E9010C94E901B000000002
:1000B0000004BFFF78FF000000000000F500F00022
:1000C000F4000000F200F100F300FD00FE00FF006C
:1000D000000000010101010101010101020202020F
:1000E00002020202020303030303030303040404E2
:1000F00004040404050505050506060606060707AB
:1001000007070708080808090909090A0A0A0B0B62
:100110000B0C0C0C0D0D0D0E0E0E0F0F0F10101101
:100120001111121213131414151516161717181887
:1001300019191A1A1B1B1C1D1D1E1E1F20202122EF
:1001400022232424252626272829292A2B2C2D2D35
:100150002E2F30313232333435363738393A3B3C52
:100160003D3E3F404142434445464748494A4C4D45
:100170004E4F50515354555658595A5B5D5E5F610E
:100180006264656668696B6C6D6F707273757778A1
:100190007A7B7D7E8082838587888A8C8E8F9193FF
:1001A0009596989A9C9EA0A2A3A5A7A9ABADAFB126
:1001B000B3B5B7BABCBEC0C2C4C6C9CBCDCFD1D40B
:1001C000D6D8DBDDDFE2E4E7E9EBEEF0F3F5F8FAB1
:1001D000FDFF04033000000010034C0079006E00A6
:1001E000650070006100640000000A0351005600C1
:1001F0004500580000000403090409023B00020105
:1002000000A0FA0904000001030101000921110105
:1002100000012240000705810308000A09040100CB
:10022000010300000009211101000122BC000705A3
:10023000820320000A1201100100000008565150EC
:100240004C01000102030105010902A10185020917
:1002500001A100050919012905150025019505755C
:1002600001810295017503810105010930093115EC
:1002700081257F95027508810609381581257F95AE
:100280000175088106050C0A38021581257F950144
:1002900075088106C0C005010980A1018503190107
:1002A0002AB700150126B700950175108100C00519
:1002B0000C0901A101850419012AA002150126A03B
:1002C00002950175108100C005010906A10185058F
:1002D000050719E029E71500250195087501810238
:1002E0000507190029EF1500250195F07501810218
:1002F00005081901290595057501910295017503F8
:100300009101C005010906A101050719E029E715BA
:100310000025019508750181029501750881010587
:1003200007190029FF150026FF00950675088100B2
:1003300005081901290595057501910295017503B7
:100340009101C00011241FBECFEFDAE0DEBFCDBFA8
:1003500004B603FE27C080919A0290919B02A0915F
:100360009C02B0919D028730904BA740B04BD1F4D6
:1003700010929A0210929B0210929C0210929D027F
:1003800014BE84B7877F84BF0FB6F894A895809178
:100390006000886180936000109260000FBEE0E012
:1003A000F8E3099511E0A0E0B1E0E4E2FAE402C06C
:1003B00005900D92A23BB107D9F722E0A2EBB1E084
:1003C00001C01D92AA39B207E1F70E940F1F0C94D9
:1003D000D4240C94000052985A983E984698549809
:1003E0005C9826982E9857985F9824982C98089592
:1003F000809116019091170190931501809314013B
:1004000089B182FB882780F9809316011092170129
:10041000809112019091130190931101809310012A
:1004200086B186FB882780F9809312011092130110
:1004300080910E0190910F0190930D0180930C011A
:1004400089B18295817080930E0110920F01809185
:100450000A0190910B01909309018093080183B1E7
:1004600086FB882780F980930A0110920B01809106
:10047000060190910701909305018093040189B1D1
:10048000082E000C990B892F881F8827881F8093BE
:10049000060110920701809102019091030190934F
:1004A00001018093000183B18295817080930201E4
:1004B000109203010C948B028CEA90E09093B601A9
:1004C0008093B50148E76FEF8FEB0C949809CF92BA
:1004D000DF92EF92FF926B017C0140E00E942516B3
:1004E000682F80E00E94120AC701B601FF90EF90CA
:1004F000DF90CF900895811106C089EF611101C08E
:100500008AEF0C94A20F813029F48AEA6111F9CFA5
:1005100089EAF7CF089580911201909113012091FB
:100520001001309111018217930729F0181619064E
:100530007CF50C94960380910E0190910F0120910F
:100540000C0130910D018217930739F01816190626
:10055000B4F089EF90E00E94000380910A0190912D
:100560000B0120910801309109018217930781F056
:10057000181619064CF08AEF90E00C94000389EFEE
:1005800090E00E941503E9CF8AEF90E00C941503E8
:100590000895CF93DF939C013A9521153F4168F56B
:1005A000EC01CC27D170DC01AA27B270AC01442742
:1005B00054709C012227387094FF11C080E1CD2B2C
:1005C00009F480E0AB2B09F08062452B09F08064D0
:1005D000232B09F08068FB01DF91CF91099481E022
:1005E000CD2B09F480E0AB2B09F08260452B09F09C
:1005F0008460232B81F38860EECFDF91CF91089543
:10060000CF93DF93EC01805E9109089720F06BE1B6
:1006100072E1209711F465EB7FE0CE010E94C902E0
:100620008C2FDF91CF910C94250FCF93DF93EC01AA
:100630000E94730FCE01805E9109089720F062E25C
:1006400072E1209711F46CEB7FE0CE01DF91CF9146
:100650000C94C90281E0089581E008950C942C0364
:1006600008950C9430031F93CF93DF9300D000D0F4
:100670000F92CDB7DEB749835A836B833091CF0198
:1006800089819A8131111DC06623B9F02223A9F016
:100690000E943E17182F682F89819A810E94EB16BD
:1006A00069817A81812F0F900F900F900F900F909A
:1006B000DF91CF911F910C94EB030E941717182F15
:1006C000EFCF0E943E1769817A81EDCFFC01262F82
:1006D000408151816281738184810C943303CF9373
:1006E000DF93EC0160E00E946603BE01DF91CF91D1
:1006F0000C9431030E94BE1A0E948818811102C016
:100700000E9425190C94F7050C94F80108950C9497
:10071000860381E008950C948903CF93C82F0E942B
:1007200087038C2FCF910C948B0308950E943F1266
:100730000E9495032FEF84E39CE02150804090407D
:10074000E1F700C000000C94AB1A0F931F93CF93F6
:10075000DF93EC0161E00E9466038C01BE010E9400
:100760002E03882359F1BE01C8010E94380C88234A
:1007700029F1BE01C8010E948A0C8823F9F0BE014C
:10078000C8010E94AD0D8823C9F0BE01C8010E94B6
:10079000340A882399F08A81882339F001158CE581
:1007A000180751F00E3D1C4579F0CE01DF91CF9135
:1007B0001F910F910C942A030E94960380E0DF9111
:1007C000CF911F910F9108950E942519F7CF90E0C6
:1007D00080E008950895E72FF0E093E0899FE00D11
:1007E000F11D1124EE0FFF1FEE0FFF1FE60FF11D8D
:1007F000EE0FFF1FE654FF4F859194910895FC0181
:10080000EE0FFF1FEE52FF4F859194910895CF9305
:10081000DF930E94EB030E941C05EC01811520E58B
:10082000920708F042C0811530E4930708F0BDC07C
:10083000883E910528F5803E910508F09DC0883AD4
:10084000910588F4853A910508F08FC081309105B3
:1008500009F492C0009709F48FC0049708F08CC087
:10086000D0E0C0E089C08F3B910508F489C0805C6E
:100870009109C03CD105A0F30E94FF03EC017CC0AC
:100880008115904250F4C11581E0D80708F074C07A
:10089000C03FD10528F3D0656FC0C11590E3D907DB
:1008A00008F079C0CE019F70E7CF811525E592074A
:1008B00058F5811534E5930708F0A6C0811542E587
:1008C000940750F4C11581E5D80708F471C0DC2FF6
:1008D000CC27C16FD06A50C0982F969596959E01EF
:1008E00023703327C115D34508F07FC0C1E0D0E0A5
:1008F00002C0CC0FDD1F2A95E2F720E2929FC001D3
:100900001124C82BD92B6FC0C11589E5D807A8F4CD
:10091000C11598E5D90708F07CC0C11526E5D207B6
:1009200008F09ECF8C2F0E94B305C82FD0E0DC2F9B
:10093000CC27CC27DF71D0621FC0C1153AE5D307A1
:1009400008F46CC0CE0190568115904208F088CF13
:100950008D2F8F710E94B30590E0982F88278827EC
:100960009F719C012C2BE901E6CFC55AD0E0C05AFB
:10097000DE4FC881D0E0D064CE01DF91CF910895E1
:10098000C85AD0E0CC0FDD1FCE5CDE4F0990D88175
:10099000C02DD464F1CFCE019927D3FF03C0EC0161
:1009A000D86CEACFEC01D06CE7CFDF70D06AE4CF2F
:1009B000CE01E4E096958795EA95E1F783702C2FB8
:1009C00026952695237090E2299F90011124382BBB
:1009D0008C2F8370C1E0D0E002C0CC0FDD1F8A9560
:1009E000E2F7C22BD32BDC68C7CFC1E0D0E002C056
:1009F000CC0FDD1F2A95E2F730E2939FC00111244E
:100A0000C82BD92BDA68B8CFD82FCC27C46FD06ABF
:100A1000B3CFDC2FCC27C06FD06AAECF8C2F8F70B6
:100A20000E94B30534E0D695C7953A95E1F7CF70AB
:100A30009C2FEC01D069A0CF82389105B1F1B0F4C0
:100A40008133910509F475C048F48932910509F4A0
:100A500069C08A32910509F473C008958533910500
:100A600009F459C08933910501F10895833E910538
:100A7000A9F138F4803E9105F9F0823E910549F1E3
:100A80000895863E9105A9F1873E9105C9F1843EFE
:100A9000910519F520918C0221FF1FC080918B02D6
:100AA00084FD14C087EE90E0089520918B0223709E
:100AB000A1F080EE90E0089520918B0220FD47C0C8
:100AC00030918C0230FF09C024FF44C090E080E0E8
:100AD00004C020918B0222FDF7CF089520918B0254
:100AE00022FD3BC030918C0230FDE3CF24FFF5CFD7
:100AF000EDCF20918B0223FFF0CF24FDE7CFD2CFA3
:100B000020918B0223FD2CC030918C0231FFEECF5F
:100B100084EE90E0089520918B0225FFDECF89E2DC
:100B200090E0089520918B0225FFD7CF85E390E0D8
:100B3000089520918B0226FFD0CF8AE290E008959D
:100B400020918B0226FFC9CF81E390E0089589E3CD
:100B500090E0089583EE90E0089582EE90E008958D
:100B600086EE90E0089590918B0292FF06C0282FA8
:100B700028712830F9F4877F846093FF06C0282FFE
:100B800028712831F1F4877E846120918C0220FF46
:100B900006C0382F38713830D9F4877F816021FF43
:100BA00006C0282F28712831D1F4877E816194FDF9
:100BB000877E0895282F24712430F9F68B7F886072
:100BC000DCCF282F2471243101F78B7E8861DDCFA3
:100BD000382F3171313019F78E7F8860E0CF282FA0
:100BE0002171213121F78E7E8861E1CF08950C9427
:100BF000F605E82FF0E0ED58FD4F80810895089547
:100C000080EA8A95F1F70895CF93DF93A7E6B1E0E4
:100C10004AE651E0C1E0D0E08D91E82FE295EF7017
:100C2000F0E061A18F709E0101C0220F8A95EAF762
:100C3000922F9095962391A382A1822B82A34A178B
:100C40005B0751F7A3E6B1E047E651E0C1E0D0E031
:100C50008D91E82FE295EF70F0E061A18F709E0119
:100C600001C0220F8A95EAF7922F9095962391A3BF
:100C700082A1822B82A34A175B0751F71092700260
:100C8000109273021092710210927402109272020A
:100C90001092750283E00E94D106DF91CF910C94EF
:100CA0007A038F929F92AF92BF92CF92DF92EF9290
:100CB000FF920F931F93CF93DF9387E6A82E81E0D7
:100CC000B82E00E712E0912CCC24C394D12CF5016E
:100CD00081915F01C82FC295CF70D0E099A18F702C
:100CE000760101C0EE0C8A95EAF7892F8E2989A337
:100CF0008AA18E2C809488218AA30E940006E3E6B4
:100D0000F1E050E040E020E03191A32FA295AF70D8
:100D1000B0E090968C9190E03F7002C095958795D9
:100D20003A95E2F780FD39C08C2D042E01C0880F62
:100D30000A94EAF7282B4F5F5F4F4430510521F7A3
:100D400089A1882289A28AA1E82AEAA2F8018081E1
:100D5000281729F1208381E0982A0F5F1F4FFAE6B8
:100D6000AF16F1E0BF0609F0B2CF292D43E063E7EB
:100D700072E080E792E00E94D2060E948403892DEF
:100D8000DF91CF911F910F91FF90EF90DF90CF9067
:100D9000BF90AF909F908F90089580E0CBCF80E080
:100DA000DBCF0895FF920F931F93CF93DF93F82E1D
:100DB000092F162FD72FC42F222349F081E08093CB
:100DC000B4010E946C1A9093B3018093B201809198
:100DD000B4018823A1F08091B2019091B3010E94E7
:100DE000781A069760F0EF2DF02FA12FBD2FCE0FB0
:100DF000DF2FD11DEC17FD0741F41092B401DF91F4
:100E0000CF911F910F91FF90089581918D93F2CF13
:100E1000EF92FF920F931F93CF93DF93EB01E82F95
:100E2000D11110C0442321F0F0E0EE52FF4FE491C5
:100E30006E2F7E2F8E2FDF91CF911F910F91FF90FC
:100E4000EF9008950D2F10E0282F30E0442329F073
:100E50002E523F4FF901249130E0F6E0CF9FC001C0
:100E60001124EFEFF0E0BF010E945524AB018C2F5D
:100E700090E0880F991FA5E5A49FB001A59F700D74
:100E80001124861B970B982F990F980FBF01601B99
:100E9000710B629FD001639FB00D729FB00D112442
:100EA0008B2F9D9FB0011124672F7727EF01C61B61
:100EB000D70BBE01629FE001639FD00D729FD00DE2
:100EC00011247F01E91AF108E09EB001E19E700D46
:100ED000F09E700D1124672F7727E61BF70BE29F1A
:100EE0008001E39F100DF29F100D1124E12F722F4E
:100EF0004230510599F048F44115510569F04130EF
:100F0000510581F0EB2F8D2F07C04430510569F05A
:100F100080F046305105B1F76E2F8DCFE22F7B2F39
:100F2000812FFACFE22F7D2FF7CFEB2F822F712F5A
:100F3000F3CF7B2F822FED2FEFCF41E00C940807EA
:100F4000CF93DF93762FE901682F842F0E949D07AE
:100F5000798368838A83DF91CF910895413F08F0B8
:100F600040EF0C94A00780917602982F9E7F71F439
:100F700080917602817082608093760280917902FE
:100F8000813F18F080EF809379020895843080F7D4
:100F9000F5CF88E090E00C949424CF92DF92EF920A
:100FA000FF926B017C010E94B307B701A60188E0A4
:100FB00090E0FF90EF90DF90CF900C94B224E6E7A2
:100FC000F2E083E0808311828FEF828380EF83835E
:100FD000148260817181828193810C94CD079091FC
:100FE0007A02933018F49F5F90937A02882351F02D
:100FF00060917602709177028091780290917902E7
:101000000C94CD07089581E00C94EF0790917A023B
:10101000992319F0915090937A02882351F06091AE
:1010200076027091770280917802909179020C9407
:10103000CD07089581E00C94060821E030E001C05E
:10104000220F8A95EAF79091BA01922381E009F480
:1010500080E0089570E00C948C0A6F927F928F92DA
:101060009F92AF92BF92CF92DF92EF92FF920F9337
:101070001F93CF93DF9300D000D00F92CDB7DEB790
:10108000709019019091760290FF26C0C090B50132
:10109000D090B601C114D10489F58091180133E0D4
:1010A000839FC0011124672D85589D4F0E942A08F7
:1010B0000F900F900F900F900F90DF91CF911F9195
:1010C0000F91FF90EF90DF90CF90BF90AF909F90E7
:1010D0008F907F906F90089580911A0120911B014D
:1010E00033E0839FF0011124E558FD4F821770F61D
:1010F0001182108212828F5F3396F8CF90FFCDCF8E
:10110000F12CE12C43E0642E8E2D0E941D088823D3
:1011100009F43CC0F701EE0FFF1FEC0DFD1DA5907B
:10112000B490A114B10409F4B8CF45E050E0B50182
:10113000CE0101960E94832409810F3F39F18A81F3
:10114000800F9927991F8530910514F084E090E075
:101150004C01880C991C880D991D9C0125583D4F08
:101160004901069D8001112405581D4F08151905D8
:1011700020F035E0A30EB11CD8CF98014D816C81D1
:101180008B810E94AE070D5F1F4FF0CF8FEFE81AE3
:10119000F80A28E0E216F10409F0B6CF7ECFE6E7C0
:1011A000F2E080818E7F8083608171818281938172
:1011B0000E94CD072FEF80E792E0215080409040C1
:1011C000E1F700C000000C942D089091760290FF8A
:1011D00014C090911A0120911B0133E0939FF001FC
:1011E0001124E558FD4F921710F00C942D088183BF
:1011F000608342839F5F3396F6CF0895EF92FF920C
:101200000F931F93CF93DF9300D00F92CDB7DEB72C
:10121000F82E062F142FE22E8091760280FF28C030
:10122000E82FE695F0E0E659FE4F90819093B801E3
:101230008E7F823059F49E012F5F3F4F8F2D0E9489
:10124000AE074B8169818A810E94E508F09277029E
:101250000093780210937902EE2051F060917602AB
:101260007091770280917802909179020E94CD0767
:101270000F900F900F90DF91CF911F910F91FF90E2
:10128000EF900895E6E7F2E09181282F4381628193
:1012900088E0890F0C94FE0881E00C944209E6E78F
:1012A000F2E09181282F4381628188EF890F0C94AD
:1012B000FE0881E00C944F09E6E7F2E0628128E045
:1012C000620F08F46FEF282F438181810C94FE0890
:1012D00081E00C945C09E6E7F2E0628128E0621BA1
:1012E00008F460E0282F438181810C94FE0881E09E
:1012F0000C946B09E6E7F2E0438128E0420F08F422
:101300004FEF282F628181810C94FE0881E00C94BC
:101310007A09E6E7F2E0438128E0421B08F440E066
:10132000282F628181810C94FE0881E00C94890948
:1013300020E00C94FE088091760280FF18C0817036
:10134000826080937602662351F0609176027091FC
:10135000770280917802909179020E94CD074091A6
:10136000790260917802809177020C94980908952F
:10137000682F81E00C949B0981E00C94B809682FD8
:101380009091760296958FEF890F09F481E00C9485
:101390009B0981E00C94BF0961E00C949B09E6E78E
:1013A000F2E080818160808386950C94CC098091E5
:1013B000760280FD0C94CF080C94CF0960E00C9469
:1013C0009B098091B70181112CC00E94881881115E
:1013D00004C00E9425190E94DF070E94C90760937C
:1013E00076027093770280937802909379026E7FF1
:1013F00061F40E94DF070E94C90760937602709330
:10140000770280937802909379020E94B3078091CB
:10141000760280FF03C086950E94DE0981E08093FA
:10142000B701089521E030E0A90102C0440F551F23
:101430008A95E2F7CA012091BA01662361F0822BF6
:101440008093BA018091B901811108C08091760220
:1014500086950C94DE0980958223F2CF0895FA01D7
:10146000811101C0FB0109940F931F93CF938C014D
:10147000FB01C281CC2309F44DC00E94D3178272B4
:10148000F801E25CFC45E431F10538F4EA52FB4D29
:101490000C947D240E94D709C0E08C2FCF911F911E
:1014A0000F91089549EC59E06CEB79E00E942F0A06
:1014B000F3CF4CEB59E069EC79E0F8CF49E559E01E
:1014C0006CE479E0F3CF4CE459E069E579E0EECFE4
:1014D00047E759E068E679E0E9CF48E659E067E791
:1014E00079E0E4CF45E959E066E879E0DFCF46E806
:1014F00059E065E979E0DACF4AE158E063E078E065
:10150000D5CF43E058E06AE178E0D0CF81E00E9497
:10151000CC09C2CFC1E0C1CF539A4BB1477F5BB179
:101520005860EFB7F8949B01220F331F260F371F27
:10153000280F391F2817390741F4EFBF8FE594E0D2
:101540000197F1F700C000000895DC016D91CD0115
:1015500078E05BB9000000C067FF4BB9660F000080
:1015600000C000C000C04BB900C07A9591F7E2CF2F
:101570000C947B02AF92BF92CF92DF92EF92FF92D8
:101580000F931F93CF93DF93AEE7B1E02CE731E0E9
:101590008FEBA82E81E0B82E60E871E041E050E0CA
:1015A0000D91802F82958F7090E0FC01C1A10F708A
:1015B0007A01002E01C0EE0C0A94EAF7FE2DF09598
:1015C000CF23FC01C1A3C2A1CE29C2A3E901199175
:1015D0009E01E12FE295EF70F0E0F1A01F706A012B
:1015E000012E01C0CC0C0A94EAF7EC2CE094EF2019
:1015F000E1A2F2A0FC28F2A2EC0188A190E002C0D6
:10160000959587950A95E2F78170E0A1F0E002C018
:10161000F595E7951A95E2F790E0E0FD92E0892BC9
:10162000F50181935F016A177B0709F0B9CFDF915C
:10163000CF911F910F91FF90EF90DF90CF90BF90CF
:10164000AF9008959F92AF92BF92CF92DF92EF92A8
:10165000FF920F931F93CF93DF930FEB11E08EE771
:10166000C82E81E0D82E9CE7E92E91E0F92E2DEBD3
:10167000A22E21E0B22ECBEBD1E0912CD801EC913F
:10168000EE0FEE0FED938D01D6012D916D01A22F7E
:10169000A295AF70B0E090968C9190E02F7002C050
:1016A000959587952A95E2F781709927D7014D91F5
:1016B0007D01A42FA295AF70B0E090962C9130E000
:1016C0004F7002C0359527954A95E2F7A901417000
:1016D000552720FF02C042E050E0842BE82BD801C0
:1016E0001197EC93EF70F0E0E459FE4F8081F50123
:1016F0009081890F808384303CF088818F5F88835C
:1017000060E0892D0E94B80AD5018C918D3F3CF490
:1017100088818150888361E0892D0E94B80AF50193
:101720008081837887FF03C081508C6F8F5FD501E4
:101730008D935D012196B1E09B120CC0DF91CF919A
:101740001F910F91FF90EF90DF90CF90BF90AF90DF
:101750009F9008959924939491CFAF92BF92CF9286
:10176000DF92EF92FF920F931F93CF93DF937C0151
:101770005B01C42FD22FFC0182818823F9F04093B2
:10178000C3010E946C1A9093C2018093C10180E250
:101790008C0F883008F061C0C77081E001C0880FED
:1017A000CA95EAF7DF91CF911F910F91FF90EF90CB
:1017B000DF90CF90BF90AF900C94B50F1091C30104
:1017C000141340C08091C1019091C2010E94781A07
:1017D0006C01B701C5010E94B514C816D90690F571
:1017E000C0E2CD0F1D17B9F080E2810F883040F4C0
:1017F000177081E001C0880F1A95EAF70E94BC0FAC
:10180000C83048F481E09D2F977001C0880F9A95E9
:10181000EAF70E94B50F802F0E94A20FC830E8F4AB
:10182000D77081E001C0880FDA95EAF7DF91CF9198
:101830001F910F91FF90EF90DF90CF90BF90AF90EE
:101840000C94BC0F80E28C0F883038F4C77081E0B4
:1018500001C0880FCA95EAF7E9CFDF91CF911F91B8
:101860000F91FF90EF90DF90CF90BF90AF900895D1
:101870000F939C01CB01233F4CE5340759F1A8F4A9
:10188000283DFCE53F0701F1293D4CE53407D1F146
:10189000273D3C4591F406E221EE41EE67ED7CE503
:1018A0000E94AD0B80E00F910895253FFCE53F07B6
:1018B000E9F0B0F0263F3C45F9F0FC018281882335
:1018C00039F11092C301EFCF07E225EE45EE68ED46
:1018D0007CE5E6CF06E221EE40EE63EF7CE5E0CF6B
:1018E00007E225EE44EE64EF7CE5DACF06E221EE76
:1018F00042EE65EF7CE5D4CF07E225EE46EE66EFDB
:101900007CE5CECF08E221E045EE69ED7CE5C8CF6D
:1019100081E0C9CFCF93DF93EC01FB018281882363
:1019200009F419C1C230FCE5DF07C0F1C6319CE5FE
:10193000D90730F09E012A5F3C452930310570F50A
:101940000E949B1890938C0280938B02C031ECE52F
:10195000DE0709F4CFC008F05BC0C8308CE5D807BB
:1019600009F4B6C088F5C430ECE5DE0709F4A8C078
:10197000C0F4C2308CE5D80709F49CC080918B027A
:101980008260C330DC4509F498C080918B0290914D
:101990008C020E94A9180E943F1280E0DF91CF9133
:1019A000089580918B028061C630ECE5DE0709F472
:1019B00084C080918B028860C730DC4508F47DC00C
:1019C00080918B02806279C0CC308CE5D80709F415
:1019D00089C070F480918B028C60CA30ECE5DE0720
:1019E00009F46BC008F478C080918B028E7F65C0CB
:1019F000CE308CE5D80709F479C080918B028B7FBB
:101A0000CF30DC4508F459C080918B028F7E55C0E1
:101A1000CB3FECE5DE0709F457C030F5C3318CE568
:101A2000D80709F46FC078F4C131ECE5DE0709F49A
:101A300065C0C231DC4509F0A8CF0E943F128091F9
:101A40008B028F773AC0C5318CE5D80709F462C0A4
:101A500008F476C080918C028160CA3FDC4509F0B1
:101A600094CF80938C0291CFCF3FFCE5DF0709F440
:101A70004DC088F480918C028D7FCD3F9CE5D907C5
:101A800081F380918C028E7FCE3FDC4550F38091B4
:101A90008C028360E6CFC130FDE5DF0709F459C051
:101AA00008F444C080E0C230DD4509F06ECF0E94EA
:101AB00027196BCF80918B02816080938B0265CF59
:101AC00080918B028460F9CF80918C028260C9CFB3
:101AD00080918B028064F1CF0E943F1280918B0233
:101AE0008068EBCF80918B028D7FE7CF80918B0256
:101AF000877FE3CF80918B028F7DDFCF80918B0238
:101B00008F7BDBCF80918B02837FD7CF80918C023C
:101B10008C7FA7CF80918B0282FB992790F921E0DF
:101B2000922790FB82F990FB83F9C7CF80918C02BA
:101B3000982F909591708E7F892B90FB81F991CF92
:101B40000E943F1290918B02892F97FB87F9805852
:101B5000B4CF81E0ACCF81E021CFCF93DF93EB0115
:101B600086319C4511F50E94D3179A81992399F0EB
:101B70008A7A91E009F490E09093C401811109C040
:101B800089E20E94AE170E941F1880E0DF91CF917A
:101B9000089585E3F6CF8091C401811104C089E2E4
:101BA0000E94B517F0CF85E3FBCF81E0EFCF909394
:101BB000CA018093C9010895E091C901F091CA0159
:101BC000309721F00190F081E02D099480E0089594
:101BD000E091C901F091CA01309799F0209131014B
:101BE000222359F020918B0227FF07C0DC012C91A2
:101BF00011962C93119725E02C930280F381E02D10
:101C000009940895E091C901F091CA01309739F023
:101C100022E0DC012C930480F581E02D09940895E5
:101C20002091C7013091C8012817390771F09093AE
:101C3000C8018093C701E091C901F091CA013097B2
:101C400021F00680F781E02D099408952091C501C7
:101C50003091C6012817390771F09093C60180931F
:101C6000C501E091C901F091CA01309721F00084CB
:101C7000F185E02D0994089585B7806885BF85B703
:101C8000806885BF089508950C945C020E943C0E04
:101C90000E94430E0C94EB0181E008950C944C0ECD
:101CA0000E94631A0E9404060E94D51A0E94E1094C
:101CB0000E94BA0A0C94440EBF92CF92DF92EF9228
:101CC000FF920F931F93CF93DF93CDB7DEB72A9781
:101CD0000FB6F894DEBF0FBECDBF0E9451060E9422
:101CE0004E0E882309F461C08CECC82E81E0D82EFA
:101CF00010E000E0B02E802F0E94F905E82EF601DA
:101D0000F1906F01F81609F44AC080913F0281FDFD
:101D10000E94FF059F2D9E2580E0FF24F394292F2C
:101D20002F21C1F18E83BF82EF2081E009F480E092
:101D300088870E946C1A8160782F9A8789874E81E4
:101D40005F8168858A850E94F60EF801E453FE4F94
:101D50008081F826F0820E94220B0E94801C0E9443
:101D6000DC0D9091CB01891789F10E94DC0D8093E5
:101D7000CB012A960FB6F894DEBF0FBECDBFDF9120
:101D8000CF911F910F91FF90EF90DF90CF90BF9078
:101D90000C948D038F5FFF0C843009F0C0CF0F5F70
:101DA0001F4F0330110509F0A5CF8FEF89838A8378
:101DB0001B820E946C1A8160782F9D838C834981DD
:101DC0005A816B818D810E94F60EC5CF2A960FB67F
:101DD000F894DEBF0FBECDBFDF91CF911F910F9161
:101DE000FF90EF90DF90CF90BF900895CF93DF9357
:101DF000CDB7DEB72B970FB6F894DEBF0FBECDBFC1
:101E00004F83588769877A878B871E821D8285E07A
:101E1000FE013796DE01119601900D928A95E1F749
:101E200049815A816B817C818D819E812B960FB671
:101E3000F894DEBF0FBECDBFDF91CF910C94B814E4
:101E4000FC01808191810C948017CF93C82F882347
:101E500009F447C08CEF8C0F813AA0F46C2F80916D
:101E60001D0190911E010E944019882329F08C2F9A
:101E70000E94B5170E941F188C2F0E94AE17CF9199
:101E80000C941F1880E28C0F883048F4C77081E0F2
:101E900001C0880FCA95EAF70E94D617F0CFEBE58C
:101EA000EC0FE33040F4F0E0E255FE4F808190E02B
:101EB000CF910C94100EE8E5EC0FE73150F4F0E010
:101EC000EE0FFF1FE058FE4F80819181CF910C945F
:101ED000260EC03F30F08C2F0E947A1BCF910C94BD
:101EE000651CCF910895882361F19CEF980F913A7A
:101EF00020F40E94B5170C941F1890E2980F9830A8
:101F000050F4877091E001C0990F8A95EAF7892F04
:101F10000E94DC17F0CF9BE5980F933020F490E0FF
:101F200080E00C94100E98E5980F973120F490E023
:101F300080E00C94260E803F20F00E94E21B0C945F
:101F4000651C0895CF93C82F0E94250FC93349F40B
:101F50002FEF87EE93E0215080409040E1F700C0E2
:101F600000008C2FCF910C94730F882321F00E94D6
:101F7000D6170C941F180895882321F00E94DC17AF
:101F80000C941F180895BF92CF92DF92EF92FF92A8
:101F90000F931F93CF93DF936C01D62FC72FFC01B4
:101FA000058102950F70128111110E94F3170E9492
:101FB000CC17E82E882391F01123D1F08C2F807F4D
:101FC000803421F080E28D0F883090F082E00E9412
:101FD0006A180E94CC1791E0E82EE926BC2EB29434
:101FE0009FE0B922EB2DF0E0E651FB4D0C947D24EF
:101FF000E12CF4CF0C2F0F70C07F11F00295007F01
:102000001123A9F0002359F080E28D0F883010F0E1
:10201000D11109C0802F0E94D6170E941F188D2F42
:102020000E94250F14C0802F0E94E617F6CF8D2F37
:102030000E94730F002359F080E28D0F883010F05A
:10204000D1112CC0802F0E94DC170E941F182B2D4D
:102050002850330B2430310520F40E94DC0D0E94FF
:102060008D03EE2009F49EC10E94C81780FD9AC11D
:10207000F60112820E94C2170E944F16C6010E94EA
:10208000F3110E94C217DF91CF911F910F91FF9022
:10209000EF90DF90CF90BF900C947016802F0E942D
:1020A000EC17D3CFFC2FFF70FF2EC07FC03219F08A
:1020B000F29480EFF822DD2369F0D13049F1112349
:1020C00091F1002351F1F601858180FFA8CF8F7037
:1020D000858323C0112381F0011106C00E940618D8
:1020E0008F290E94B50FB3CF0130C1F70E940618A7
:1020F0008F290E940C18ABCF011106C00E94151841
:102100008F2D0E94BC0FA3CF013009F4A0CFF6CFD2
:10211000112329F0063008F09ACF8F2DE2CF053039
:1021200008F095CFEDCF002359F3D93349F4FFEFF1
:1021300027EE33E0F15020403040E1F700C00000CE
:102140008D2F0E94730F83CF8C2F86958695837079
:1021500069F0813009F07BCF8D2F9C2F9370111186
:1021600002C090E080E00E94260E71CF8D2F9C2F40
:102170009370111102C090E080E00E94100E67CFB2
:102180008D2F112329F00E947A1B0E94651C5FCFBE
:102190000E94E21BFACF8C2F837009F041C011110D
:1021A00056CF4D2F429546954770440F440F0D2F43
:1021B0000F7010E030E020E0042E04C0000F111F6B
:1021C000221F331F0A94D2F760E070E0CB01D4FFE6
:1021D0000FC06FE070E080E090E004C0660F771FF2
:1021E000881F991F4A95D2F76095709580959095B4
:1021F000C695C695C370602B712B822B932BC23072
:1022000049F058F4C13019F00E94EE1520CF0E9419
:10221000DC151DCF0E9400161ACF0E94DA1517CFC9
:102220008695112311F08C2F8170882309F40FCF2C
:102230004D2F429546954770440F440F0D2F0F7058
:1022400010E030E020E0042E04C0000F111F221F18
:10225000331F0A94D2F760E070E0CB01D4FF0FC0C7
:102260006FE070E080E090E004C0660F771F881F89
:10227000991F4A95D2F76095709580959095C6956F
:10228000C695C370602B712B822B932BC23049F003
:1022900058F4C13019F00E94C616D9CE0E94B41667
:1022A000D6CE0E94D816D3CE0E941416D0CECF70B0
:1022B000112329F08C2F0E944F168D2F12CF8D2FB6
:1022C0000E94BC0F8C2F0E947016C1CED23F89F1A4
:1022D00060F4D03FC9F0D13F29F1112309F442C085
:1022E00001119DCE8C2F8F7121C0D33F39F1D43F86
:1022F000A1F7112369F1CF718C2F0E944F1663E073
:102300008C2F0E945518A3CE112341F0053008F000
:102310009ECE8C2F8F710E94931699CE063008F0B6
:1023200096CEF7CF8C2F8F71112369F20E944F1632
:102330008ECE8C2F8F711123C9F3C5CF112329F0B5
:102340008C2F8F710E943A1682CE0E9420167FCE6B
:1023500081E00E946A18023008F479CE82E00E947F
:102360006A1875CE002359F0D93309F0E9CE8FEF02
:1023700097EEE3E081509040E040E1F7DFCE8C2F14
:102380008F71A1CF4C2F4F706D2FC6010E94E703B4
:102390000E9452155CCE4C2F4F706D2FC6010E94CB
:1023A000EA0355CEDF91CF911F910F91FF90EF90EF
:1023B000DF90CF90BF9008950F931F93CF93DF933B
:1023C000EC01688179818A810E948A178C010E94C0
:1023D000EA160E94D915B801CE01DF91CF911F9165
:1023E0000F910C94C30FCF93DF93EC018B819C81F1
:1023F000892B29F08881998189238F3F59F4DF91B6
:10240000CF910895CE010E94DC11CE01DF91CF91D2
:102410000C946F03CE010E94A5038111F3CF0E949B
:10242000CC17882361F38A81882349F382E0DF9106
:10243000CF910C946A18882321F00E94E6170C941F
:102440001F180895882321F00E94EC170C941F1880
:1024500008950E94F3170E9403180E941F180E94FB
:102460008C1D0E94651C90E080E00E94100E90E0A0
:1024700080E00C94260E0E94BC170C9429120E9436
:10248000E3170C943B12E92FE295EF70E250EE3027
:1024900070F4F0E0E650FB4D0C947D24803F19F081
:1024A00020F4883E20F481E00895843FE1F380E049
:1024B0000895883EC0F3813FD1F7F5CF93FB88277D
:1024C00080F908950E9480170C944312CF93DF93F4
:1024D00000D000D00F92CDB7DEB70F900F900F90C5
:1024E0000F900F90DF91CF910895CF93DF9300D09D
:1024F00000D000D0CDB7DEB726960FB6F894DEBF79
:102500000FBECDBFDF91CF9108951F93CF93DF937F
:10251000C091D00116E08091D1018C1304C0DF91ED
:10252000CF911F910895D0E01C9FF0011D9FF00DE9
:102530001124EE52FE4F408151816281738184816A
:1025400095810E9475122196C770E5CF40910202D5
:10255000509103026091040270910502809106027D
:10256000909107020C9475121F93CF93DF93809183
:102570000702807FA9F480910402882389F080916A
:10258000D001C091D1016091020270910302A0912B
:102590000502B0910602D62FD72316E0C81304C057
:1025A000DF91CF911F91089590E0109711F0DF3FD8
:1025B00019F401968770F2CF189F9001199F300D82
:1025C0001124F901EE52FE4F41814713F2CF4081B1
:1025D0004613EFCF42814111ECCF438154814A1B16
:1025E0005B0B483C510528F7809107028F70806192
:1025F00080930702F901E952FE4F80818F7080615C
:10260000808382E092E00E94F311DF91CF911F91CD
:102610000C948512AF92BF92CF92DF92EF92FF920D
:102620000F931F93CF93DF93CDB7DEB761970FB6AC
:10263000F894DEBF0FBECDBF8C0185E0F801DE014E
:102640001D9601900D928A95E1F7F8014081518124
:10265000E28082E0C82E82E0D82E6091050270915F
:1026600006026115710509F461C190910202209181
:102670000302892F82238F3F09F458C1A380B480BD
:10268000F0900402F501E61BF70BFF2009F4FCC0F3
:1026900080910702382F307FE83CF10508F0B2C086
:1026A000311179C0FE2C251323C0941321C0E110F1
:1026B0001FC08F708061809307020E94A612C6011E
:1026C0000E94F31180910702F80185838F2D619696
:1026D0000FB6F894DEBF0FBECDBFDF91CF911F9133
:1026E0000F91FF90EF90DF90CF90BF90AF90089543
:1026F000AB2829F0842F85238F3F09F033C180E078
:10270000F82FF170DF2E80FF3CC08091D001209126
:10271000D10136E0821315C04D875E878D859E8579
:102720000E948017292F22952F702230F0F024303C
:1027300018F59F70F1F0F8019581907FD1F4D12CBC
:102740001EC090E0389FF001399FF00D1124EE5229
:10275000FE4F6181651306C06081641303C062810E
:102760006E110FC001968770D5CF9F7011F088232E
:1027700031F3805E883018F3C8010E94F311FD2CFC
:10278000A5CFEE2009F4A2CF80910702816080934B
:102790000702F12C9BCF251306C0941304C0F80147
:1027A000EE2009F48DC04D875E878D859E850E9441
:1027B0006212882319F1EE2009F18091070280321C
:1027C00070F0209102023091030238872F8319861E
:1027D000BB86AA868C87CE0107960E94F31186E0FD
:1027E000F801A2E0B2E001900D928A95E1F70E9413
:1027F000B4120E94A612FF24F39468CFC8010E946D
:10280000F311F9CF311113C07A2DB98AA88A6E2D30
:1028100089890E94661282E092E00E94F31186E0AC
:10282000F60111928A95E9F70E94A612B2CF2513FC
:102830000FC094130DC0E1100BC0F8018583C801CF
:102840000E94F31186E0F60111928A95E9F73ECFD6
:102850004D875E878D859E850E946212882371F266
:10286000EE2061F280910702803208F4B8CF209107
:102870000202309103023A8329831B82BD82AC821B
:102880008E83CE010196A9CFE83CF10508F041C046
:10289000FE2CEE2009F4B2CF25132AC0941328C0D1
:1028A0008091070280FD1BC0982F907FC1F0F80136
:1028B0008583903F31F0982F907F905F8F70892BA8
:1028C0008583C8010E94F31186E0F801A2E0B2E01E
:1028D00001900D928A95E1F70E94A612F7CE86E04C
:1028E000F801A2E0B2E001900D928A95E1F7EECEF8
:1028F0004D875E878D859E850E94621281116FCF04
:1029000080910702816080930702C8010E94F31141
:10291000DDCE7A2DB98AA88A6E2D89890E94661229
:1029200086E0F60111928A95E9F7D6CFEE2009F4F8
:1029300065CF4D875E878D859E850E946212F82E39
:10294000882309F45BCF86E0F801A2E0B2E00190B1
:102950000D928A95E1F782E092E00E94200F0E949A
:10296000B412BACF81E08E25CBCE88EC90E00895EA
:102970001F93CF93DF93CDB7DEB72C970FB6F894A4
:10298000DEBF0FBECDBF4F83588769877A878B879D
:102990009C87CE0107960E940A13882369F08A85D6
:1029A0009B85892B39F04F815885842F85238F3F54
:1029B00009F071C016E05FC086E0FE013796DE01C7
:1029C000119601900D928A95E1F78A859B85892B56
:1029D00089F38F81988589238F3F61F32091D101FD
:1029E00030E0C9010196877099274091D0014817BE
:1029F000190671F40E943F121092D1011092D00179
:102A000086E0E2E0F2E0DF011D928A95E9F7D2CF9D
:102A100096E0929FD001939FB00D1124AE52BE4F0D
:102A2000FE01319601900D929A95E1F78093D101C4
:102A30000E948512BFCF819FC00111248E529E4FEC
:102A40000E940A138823E9F0E091D0011E9FF00153
:102A50001124EE52FE4F4081518162817381848145
:102A600095810E9475128091D00190E00196877047
:102A700099278093D0018091D0019091D101891341
:102A8000DACF2C960FB6F894DEBF0FBECDBFDF9124
:102A9000CF911F91089569857A858B859C850E94C9
:102AA000751288CFEF92FF920F931F93CF93DF930E
:102AB0008C01892B81F0F12CEE24E394E80121961E
:102AC000F8018491843770F4843008F05FC081305D
:102AD000B1F08230A1F1DF91CF911F910F91FF9062
:102AE000EF900895853709F44CC008F43DC09CE789
:102AF000980F903780F78F770E94730F49C00E5F51
:102B00001F4FFE01849190E2980F983060F4877017
:102B1000FE2D01C0FF0F8A95EAF78F2F0E94F6174E
:102B20000E941F1802C00E94250F8F2D815030F285
:102B3000EFE9FFE03197F1F700C00000F7CF0E5F3B
:102B40001F4FFE01849190E2980F983050F48770E7
:102B5000FE2D01C0FF0F8A95EAF78F2F0E94FC1708
:102B6000DFCF0E94730FE1CF0E5F1F4FFE01C491B4
:102B7000C150D8F28FE99FE00197F1F700C0000043
:102B8000F7CF0E5F1F4FFE01F490CFCF0E94250FAD
:102B90008E01CBCF08950C94CA150E94CB1560937B
:102BA00016027093170280931802909319020C94E6
:102BB000291208950C94CD150F931F9300911602BE
:102BC000109117022091180230911902602B712B7D
:102BD000822B932B1F910F910C94CD150F931F9364
:102BE00000911602109117022091180230911902DB
:102BF00060237123822393231F910F910C94CD1591
:102C00000F931F9300911602109117022091180242
:102C10003091190260277127822793271F910F9106
:102C20000C94CD150C9467020E9412166093120248
:102C30007093130280931402909315020C9429123E
:102C400060E070E0CB010C941416611571058105EC
:102C5000910529F481E0442361F080E00895DC01CE
:102C6000CB0104C0B695A795979587954A95D2F75D
:102C7000817008950F931F9341E050E060E070E091
:102C80008A019B0104C0000F111F221F331F8A9568
:102C9000D2F7C901B8011F910F910C9414160F932C
:102CA0001F9341E050E060E070E004C0440F551F06
:102CB000661F771F8A95D2F78091120290911302B6
:102CC000A0911402B09115028A019B01082B192BC7
:102CD0002A2B3B2BC901B8011F910F910C9414169C
:102CE0000F931F9341E050E060E070E004C0440F98
:102CF000551F661F771F8A95D2F7CB01BA016095E1
:102D00007095809590950091120210911302209178
:102D100014023091150260237123822393231F91A3
:102D20000F910C9414160F931F9341E050E060E054
:102D300070E004C0440F551F661F771F8A95D2F7B5
:102D40008091120290911302A0911402B091150289
:102D50008A019B01082719272A273B27C901B801A7
:102D60001F910F910C9414160F931F930091120250
:102D7000109113022091140230911502602B712BD7
:102D8000822B932B1F910F910C9414160F931F936A
:102D90000091120210911302209114023091150239
:102DA00060237123822393231F910F910C94141697
:102DB0000F931F930091120210911302209114029D
:102DC0003091150260277127822793271F910F9159
:102DD0000C9414160895990F990F890F982F9770D6
:102DE00041E001C0440F9A95EAF78695869586954D
:102DF00095E0899FF0011124E85FFD4F30E020E06D
:102E000070E05191DF011197CB01022E02C096951F
:102E100087950A94E2F78170819585278423852719
:102E20008C932F5F3F4F2530310559F70895990F47
:102E3000990F890F982F977086958695869525E02E
:102E4000829FF0011124E85FFD4F50E040E080E0F8
:102E5000219130E0092E02C0369527950A94E2F7B9
:102E600021703327042E01C0220F0A94EAF7822B27
:102E70004F5F5F4F4530510559F70895BF92CF928C
:102E8000DF92EF92FF920F931F93CF93DF938C010A
:102E9000C0901202D0901302E0901402F09015023C
:102EA0008091160290911702A0911802B091190218
:102EB000C82AD92AEA2AFB2ACFE1D0E0BC2ED701C2
:102EC000C6010C2E04C0B695A795979587950A94D0
:102ED000D2F780FD0EC0219788F7B12C8B2DDF91A2
:102EE000CF911F910F91FF90EF90DF90CF90BF9007
:102EF0000895B8018C2F0E940704019761F3EECF6B
:102F0000CF93DF93EC010E943E17BE01DF91CF917A
:102F10000C9407041F93CF93DF93EB019091CF01A3
:102F2000992331F0CB01DF91CF911F910C94801741
:102F3000882379F0CB010E943E17182F682FCE010D
:102F40000E94EB16BE01812FDF91CF911F910C944F
:102F50000704CB010E941717182FF4CF682F809118
:102F60001D0190911E010C94C019682F80911D01C4
:102F700090911E010C94CB1980911D0190911E011E
:102F80000C94D61980911A0285958595859508959A
:102F900080911A028770089590911A02977081E0CB
:102FA00009F480E0089580913E02089590913E02D8
:102FB000892B80933E020895809590913E0298233C
:102FC00090933E02089510923E02089590913D0222
:102FD000892B80933D020895809590913D0298231E
:102FE00090933D02089510923D02089590913C0205
:102FF000892B80933C020895809590913C02982300
:1030000090933C02089510923C02089580911B0217
:10301000089508950C94091890911B02981721F0B7
:1030200080931B020C940A18089580911B02882338
:1030300029F010921B0280E00C940A180895E09188
:103040001D01F0911E0180913E028083E0911D01DF
:10305000F0911E01808190913D02892B8083E09147
:103060001D01F0911E01808190913C02892B80838B
:1030700090911B02992381F0E0911D01F0911E01B6
:103080008081892B808380911D0190911E010E9477
:103090002C1981110E94151880911D0190911E011B
:1030A0000C94E80D08950C94521898E0899F9001B3
:1030B0001124622B60931A020E944F1680911A020B
:1030C0008595859585950C94531810921A0280E089
:1030D0000C94531890911A028095892380931A02B8
:1030E000282F277071F4282F082E000C330B92170D
:1030F000130639F08595859585950E9470160C9478
:10310000651808956FEF7FEF90E080E00C94BE2487
:1031100090E080E00E949A2421E08C3E9E4F09F0CE
:1031200020E0822F089582E090E00C948C2483E0CC
:1031300090E00C948C24CF9384E090E00E948C2447
:10314000C82F81E290E00E948C24982F8C2FCF9181
:103150000895CF93C92F682F84E090E00E94A024A7
:103160006C2F81E290E0CF910C94A024AB01BC01C4
:103170008FE090E00C94B224AB01BC0183E190E0BD
:103180000C94B22460E070E0CB010C94BC1860E0B9
:1031900070E0CB010E94B6180C94C2186CEE7EEF62
:1031A00090E080E00E94BE2460E082E090E00E9417
:1031B000A02460E083E090E00E94A0241092160218
:1031C00010921702109218021092190260E084E027
:1031D00090E00E94A02460E081E290E00E94A024A0
:1031E00060E085E090E00E94A02460E086E090E04E
:1031F0000E94A0246FEF87E090E00E94A02440E0AE
:1032000050E0BA0188E090E00E94B22460E08DE0D6
:1032100090E00E94A02440E050E0BA0188E190E0F4
:103220000E94B22460E087E190E00E94A02440E088
:1032300050E0BA018CE190E00E94B22460E080E2AC
:1032400090E00E94A0240C94C7180C94CE18682F0C
:103250008EE090E00C94A024FC0132968091310124
:10326000882321F080918B029EE187FF96E080E029
:10327000915008F4089521912223D1F38F5FF8CF64
:10328000662301F1209131012223F1F020918B027C
:1032900027FF1AC0462F4695469546954E3190F425
:1032A000677021E030E002C0220F331F6A95E2F719
:1032B000840F911DFC01828190E02823392381E055
:1032C000232B69F480E00895FC0132960896219141
:1032D000261721F0E817F907D1F7F4CF81E0089518
:1032E0009C01FC0132969FEF80E04191461751F01E
:1032F0009F3F19F4411101C0982F8F5F8630A9F7C5
:103300009F3F09F40895290F311D97FD3A95F90162
:1033100062830895FC01329608962191261303C01A
:10332000DF0111971C92E817F907B9F70895E62F06
:10333000E695E695E695EE3168F4E80FF92FF11D74
:10334000677021E030E001C0220F6A95EAF78281C0
:10335000822B82830895E62FE695E695E695EE3179
:1033600070F4E80FF92FF11D677021E030E001C023
:10337000220F6A95EAF720958281282322830895F7
:1033800020913101222329F020918B0227FD0C94FA
:1033900097190C94701920913101222329F0209162
:1033A0008B0227FD0C94AB190C948A19FC01329600
:1033B00080913101882351F080918B0287FF06C0F4
:1033C0008EE1DF011D928A95E9F7089586E0F9CF35
:1033D000089508950C94E9190E94EA1980919102C8
:1033E000843049F11092400288E190E020E40FB669
:1033F000F894A895809360000FBE2093600080E051
:103400000E948D030E94EA1983B7817F846083BF85
:1034100083B7816083BF7894889583B78E7F83BF9D
:103420000FB6F894A8958091600088618093600041
:10343000109260000FBE08950895CF930E94E8197E
:103440000E9451060E941C1AC0E08C2F0E94F905B0
:10345000811105C0CF5FC330C1F7CF91089581E0DE
:10346000FCCF08950C94311A0E943F120E94DC0D8B
:103470000E948D030C94321A1F921FB61F921124C2
:103480008F939F93AF93BF9380914002811113C09C
:103490008091870290918802A0918902B0918A025E
:1034A0004196A11DB11D8093870290938802A0933D
:1034B0008902B0938A02BF91AF919F918F911F9023
:1034C0001FBE1F90189582E084BD93E095BD9AEFD2
:1034D00097BD80936E0008952FB7F894809187026E
:1034E00090918802A0918902B0918A022FBF08951D
:1034F0009C014FB7F8948091870290918802A09127
:103500008902B0918A024FBF821B930B0895789471
:103510001F921FB61F9211248F939F93AF93BF9357
:103520008091870290918802A0918902B0918A02CD
:103530000196A11DB11D8093870290938802A093EC
:103540008902B0938A02BF91AF919F918F911F9092
:103550001FBE1F90189587E797E790930108809307
:10356000000888E19AE00FB6F894A895809360006F
:103570000FBE90936000FFCF0C9482180E945106FA
:103580002FEF86E791E0215080409040E1F700C0A6
:1035900000000E94510680E00E94F90580FF04C0EF
:1035A0000E94BC1A0C94AB1A08950E9488188111CD
:1035B00002C00E9425190E94931880933F020E9426
:1035C0009B1890938C0280938B020E949718682F0F
:1035D00070E090E080E00E94DA1560911202709134
:1035E000130280911402909115020C94121680918E
:1035F000470280FF12C06091240185E0689FB001FE
:103600001124759567957595679560387105A8F5CE
:1036100061157105A1F1862F089581FF09C06091A0
:10362000240185E0689FB001112475956795EDCF61
:103630006091240182FD0AC0809146028823D1F066
:103640009091230160912401891728F085E0689FFB
:10365000B0011124DACF869FB001112485E0869F46
:103660009001879F300D1124692F70E0C9010E94DD
:103670006924CBCF65E070E0CECF8FE7089581E07D
:1036800008958091470280FF0CC06091200170E096
:1036900075956795759567956115710549F1862F43
:1036A000089581FF06C06091200170E075956795CF
:1036B000F3CF6091200182FD0BC0909145029923C8
:1036C000A1F060911F0180912001961738F0682FBA
:1036D00070E06038710500F38FE70895899FC0019D
:1036E000112470E00E946924F4CF61E070E0D7CF2C
:1036F00081E00895803F31F40E94F71A819580930C
:103700004B020895813F19F40E94F71AF8CF823FC7
:1037100031F40E94F71A819580934A020895833FFD
:1037200019F40E94F71AF8CF893F29F40E94411B2F
:1037300080934C0208958A3F21F40E94411B819599
:10374000F7CF8B3F31F40E94411B819580934D024E
:1037500008958C3F19F40E94411BF8CF843F31F447
:10376000809149028160809349020895853F21F448
:10377000809149028260F7CF863F21F4809149020F
:103780008460F1CF873F21F4809149028860EBCFBC
:10379000883F21F4809149028061E5CF8D3F31F46B
:1037A0008091470281608093470208958E3F21F403
:1037B000809147028260F7CF8F3FB9F7809147022F
:1037C0008460F1CF90914A02803F59F480914B027E
:1037D00087FF0DC010924B0291110BC01092460250
:1037E00008C0813F81F480914B0218169CF3992305
:1037F00081F080914C0290914D02892B09F064C0B8
:10380000109245020895823F49F497FFF0CF10923D
:103810004A0280914B028111ECCFE0CF833F19F433
:103820001916ACF3E4CF20914C02893F29F412160B
:10383000F4F610924C02DBCF8A3F19F427FFD7CF62
:10384000F8CF20914D028B3F29F427FFD0CF109263
:103850004D02CDCF8C3F19F41216CCF3C8CF843F64
:1038600031F4809149028E7F80934902C0CF853F19
:1038700021F4809149028D7FF7CF863F21F480911A
:1038800049028B7FF1CF873F21F480914902877FE6
:10389000EBCF883F21F4809149028F7EE5CF8D3FA9
:1038A00031F4809147028E7F80934702A0CF8E3FF4
:1038B00021F4809147028D7FF7CF8F3F09F097CF9A
:1038C000809147028B7FF0CF08950E946C1A9C0173
:1038D00090914A0280914B02982B21F03093440240
:1038E0002093430290914C0280914D02982B21F03D
:1038F000309342022093410288E492E00C94020E3D
:10390000EF92FF920F931F93CF93DF9300D000D0DD
:1039100000D0CDB7DEB786E0E8E4F2E0DE01119634
:1039200001900D928A95E1F7E0904A02F0904B02E7
:1039300000914C0210914D0210924A0210924B02DB
:1039400010924C0210924D028E2D8F2991F0809191
:103950004302909144020E94781AAC019091460271
:10396000992309F43FC0809125018417150608F4B6
:1039700047C0802F812B91F08091410290914202AB
:103980000E94781AAC0190914502992309F477C0FE
:10399000809121018417150608F47FC080914A02A6
:1039A00090914B02892B90914C02892B90914D0262
:1039B000892B11F00E94651C86E0FE013196A8E477
:1039C000B2E001900D928A95E1F726960FB6F89431
:1039D000DEBF0FBECDBFDF91CF911F910F91FF9042
:1039E000EF900895209126018AE0289F90011124EC
:1039F0002417350708F0BDCF9F5F9093460202C0A1
:103A00009F3FD1F7EE2059F00E94F71A9FEF1E1446
:103A10000CF491E0899F802D112480934A02FF20AD
:103A200059F00E94F71A9FEF1F140CF491E0899F40
:103A3000802D112480934B0230914A02332309F4E4
:103A400098CF20914B02222309F493CF45EB340306
:103A5000C0011124992359F090934A0245EB2403A5
:103A600090011124332339F030934B0282CF81E04F
:103A700080934A02F3CF81E080934B027ACF20916A
:103A800022018AE0289F900111242417350708F0AD
:103A900085CF9F5F9093450202C09F3FD1F70023DF
:103AA00059F00E94411B9FEF10160CF491E0899F82
:103AB000802D112480934C02112359F00E94411B48
:103AC0009FEF11160CF491E0899F802D11248093B3
:103AD0004D0230914C02332309F460CF20914D0206
:103AE000222309F45BCF45EB3403C0011124992351
:103AF00059F090934C0245EB240390011124332399
:103B000039F030934D024ACF81E080934C02F3CFDD
:103B100081E080934D0242CF86E0E8E4F2E0DF01ED
:103B20001D928A95E9F71092460210924502109272
:103B30004702089580916E020895CF93DF9300D0DD
:103B40000F92CDB7DEB790919102943019F5898329
:103B50007B836A8382E08093E9008FEF9091E80095
:103B6000815095FD06C095ED9A95F1F70000811101
:103B7000F5CF8091E80085FF0DC050E040E063E0A4
:103B800070E0CE0101960E94C41F8091E8008E77FC
:103B90008093E8000F900F900F90DF91CF910895E0
:103BA000BC0184E00C949D1DBC0183E00C949D1D20
:103BB0009C0182E08093E9009FEF8091E8009150A2
:103BC00085FD06C085ED8A95F1F700009111F5CFCE
:103BD0008091E80085FF0CC050E040E066E070E0B6
:103BE000C9010E94C41F8091E8008E778093E8008D
:103BF0000895CF93DF93EC01809131018823B1F1D7
:103C000080918B0287FF32C060E282E08093E900FE
:103C10008FEF9091E800815095FD06C095ED9A9543
:103C2000F1F700008111F5CF8091E80085FF1BC0FE
:103C30008091310170E050E040E0811104C050E01B
:103C400040E068E070E0CE010E94C41F8091E8006F
:103C50008E778093E80080E2FE01AEE4B2E001904E
:103C60000D928A95E1F7DF91CF91089568E081E0A8
:103C7000CDCF80919002811109C00E9454210E94F1
:103C8000B1218091E20084608093E2000895109257
:103C900090020895089508950C94341A42E061EC5E
:103CA00081E00E94D02042E261EC82E00C94D020BE
:103CB00080919302833009F45FC030F48130C1F108
:103CC000823009F49BC008958A3009F487C08B3094
:103CD00009F46DC0893009F04EC0809192028132A2
:103CE00009F049C08091960290919702029708F0DE
:103CF00042C08091E800877F8093E8008091E800CF
:103D000082FF35C09091F3008091F200029729F470
:103D10008091F1008B7F813021F48091F1008093BC
:103D20006E028091E8008B778093E8000C94042168
:103D300080919202813AF9F48091E800877F809324
:103D4000E8008091960290919702892B61F460E2DD
:103D50008EE492E070E00E9413208091E8008B775F
:103D60008093E800089560E090E080E0F3CF8091D8
:103D700091028111C3CF089580919202813AD9F7BF
:103D80008091960290919702892BA9F78091E80083
:103D9000877F8093E8008091E80080FFFCCF8091CE
:103DA00031018093F1008091E8008E77BDCF809142
:103DB0009202813201F78091960290919702892BAD
:103DC000D1F68091E800877F8093E8000E9404216B
:103DD00080919402809331010C943F128091920261
:103DE000813249F68091E800877F8093E8000E9445
:103DF00004218091950280936F0208958091920230
:103E0000813A09F0B8CF8091E800877F8093E8007D
:103E10008091E80080FFFCCF80916F02C2CF84B711
:103E2000877F84BF0FB6F894A89580916000886161
:103E300080936000109260000FBE80E890E00FB6A3
:103E4000F89480936100909361000FBE0E94460E2B
:103E50000E9454210E94B1218091E20084608093ED
:103E6000E20078940E943A240E94500E87E291E08A
:103E70000E94D70D80919102853019F00E945C0E4E
:103E8000F9CF0E94EC1980918F02882399F30E9448
:103E90001D1A882379F30E94AE1FECCF0C94501F9B
:103EA000292F33272330310519F168F421303105EA
:103EB00009F44AC02230310509F44BC090E080E09B
:103EC00030E020E028C02132310579F1223231057D
:103ED000A9F780E490E023E033E061157105D9F0A3
:103EE0008CEB90E027E432E061307105A1F0E6CF81
:103EF00099278130910599F0009741F08230910522
:103F000089F00397D9F6E2EDF1E002C0E6EFF1E0C7
:103F1000849190E09F01FA01318320830895EAEEB5
:103F2000F1E0F6CFE8EDF1E0F3CF89E090E02CE0AE
:103F300032E06115710579F389E090E025E232E025
:103F40006130710541F3BACF82E190E025E332E0C0
:103F5000E2CF8BE390E02AEF31E0DDCF80E189BD55
:103F600082E189BD09B400FEFDCF8091D8008F7D2C
:103F70008093D8008091E00082608093E00080917F
:103F8000E00081FDFCCF0895AF92BF92CF92DF9207
:103F9000FF920F931F93CF93DF936C01EB018A0184
:103FA0000E942321F82E811123C00115110539F03B
:103FB000F80180819181C81BD90BC80ED91EB12C84
:103FC000A12C2097A9F08091E80085FD22C0809166
:103FD000E8008E778093E80001151105A1F0F80143
:103FE00080819181A80EB91EB182A08285E0F82E51
:103FF0008F2DDF91CF911F910F91FF90DF90CF9088
:10400000BF90AF9008950E9423218823D1F2F82E0B
:10401000EFCFF60181916F018093F1002197FFEFBF
:10402000AF1ABF0ACECFFC018091980290919902FD
:1040300086179707A0F06115710529F49091E800A3
:104040009E779093E80090E06115710551F491110D
:1040500008C08091E80082FF34C080E00895BC0170
:10406000F2CF809191028823C1F18530C1F1809116
:10407000E80083FD30C08091E80082FDEACF8091A6
:10408000E80080FFE1CF8091F3002091F200382F0B
:104090006115710519F02830310558F091E028308C
:1040A000310509F090E02091E8002E772093E80098
:1040B000CBCF81918093F100615071092F5F3F4F09
:1040C000E7CF80919102882341F0853041F08091C3
:1040D000E80083FFBECF81E0089582E0089583E089
:1040E0000895FC0180919802909199028617970794
:1040F000A0F06115710529F48091E8008E77809316
:10410000E80090E06115710551F4911108C08091AB
:10411000E80082FF35C080E00895BC01F2CF8091B5
:1041200091028823C9F18530C9F18091E80083FDAF
:1041300031C08091E80082FDEACF8091E80080FFE5
:10414000E1CF8091F3002091F200382F61157105C5
:1041500019F02830310558F091E02830310509F088
:1041600090E08091E8008E778093E800CBCF849137
:104170008093F1003196615071092F5F3F4FE6CF78
:1041800080919102882341F0853041F08091E800D0
:1041900083FFBDCF81E0089582E0089583E0089514
:1041A000982F973028F08F708093E90081E0089570
:1041B0009093E900242F762F50E0981731F07091FA
:1041C000EC002091ED005091F00021FD02C09F5FB6
:1041D000E8CF3091EB003E7F3093EB003091ED0063
:1041E0003D7F3093ED003091EB0031603093EB0078
:1041F0007093EC002093ED005093F0002091EE00BE
:1042000027FDE5CF80E008958091920287FF13C0DB
:104210008091E80082FF06C08091E8008B77809350
:10422000E80004C0809191028111F2CF089580913D
:1042300091028823D9F38091E80080FFF8CF809124
:10424000E8008E77ECCF2091E4003091E50095E610
:10425000A9012091EC00822F817020FF06C080917F
:10426000E80080FF06C080E008952091E80022FD6C
:104270001AC080919102882389F0853089F080915D
:10428000EB0085FD0FC02091E4003091E50042175E
:104290005307F9F29150E1F684E0089582E0089521
:1042A00083E0089581E008950E94C2210E94CA21FE
:1042B000E0EEF0E0808181608083E8EDF0E08081D5
:1042C0008F77808319BCA7EDB0E08C918E7F8C93A3
:1042D00080818F7E80831092900208950F931F93A8
:1042E000CF93DF930E94C2210E94CA21C8EDD0E083
:1042F00088818F77888388818068888388818F7D93
:10430000888319BC1092910210928D0210928F0234
:1043100010928E0200EE10E0F80180818B7F808386
:1043200088818160888342E060E080E00E94D02044
:10433000E1EEF0E080818E7F8083E2EEF0E080812C
:1043400081608083808188608083F80180818E7F96
:104350008083888180618883DF91CF911F910F9145
:104360000895E8EDF0E080818F7E8083E7EDF0E056
:1043700080818160808384E082BF81E080939002AD
:104380000C946E21E8EDF0E080818E7F80831092A6
:10439000E20008951092DA001092E10008951F9251
:1043A0000F920FB60F9211242F933F934F935F9369
:1043B0006F937F938F939F93AF93BF93EF93FF93ED
:1043C0008091E10082FF0BC08091E20082FF07C074
:1043D0008091E1008B7F8093E1000E9439248091DD
:1043E000DA0080FF19C08091D80080FF15C080914D
:1043F000DA008E7F8093DA008091D90080FF96C02A
:1044000080E189BD82E189BD09B400FEFDCF81E074
:10441000809391020E94391E8091E10080FF19C0B3
:104420008091E20080FF15C08091E2008E7F809332
:10443000E2008091E20080618093E2008091D800E8
:1044400080628093D80019BC85E0809391020E941D
:104450004B1E8091E10084FF2BC08091E20084FF1D
:1044600027C080E189BD82E189BD89B5982F91700F
:1044700080FFFBCF8091D8008F7D8093D800809102
:10448000E1008F7E8093E1008091E2008F7E809337
:10449000E2008091E20081608093E20080918D02D1
:1044A000882309F449C084E0809391020E944C1E45
:1044B0008091E10083FF29C08091E20083FF25C045
:1044C0008091E100877F8093E10082E080939102F8
:1044D00010928D028091E1008E7F8093E1008091A7
:1044E000E2008E7F8093E2008091E2008061809301
:1044F000E20042E060E080E00E94D0208091F00085
:1045000088608093F0000E944A1EFF91EF91BF9156
:10451000AF919F918F917F916F915F914F913F915B
:104520002F910F900FBE0F901F90189519BC1092ED
:1045300091020E94471E70CF8091E30087FD93E0B7
:1045400090939102B3CF1F920F920FB60F92112446
:104550002F933F934F935F936F937F938F939F938B
:10456000AF93BF93CF93DF93EF93FF93D091E90085
:10457000DF708091EC00C82FC17080FDC0E8109200
:10458000E9008091F000877F8093F00078940E948A
:10459000E7221092E9008091F00088608093F0009B
:1045A000CD2BCF70C093E900FF91EF91DF91CF91B8
:1045B000BF91AF919F918F917F916F915F914F913B
:1045C0003F912F910F900FBE0F901F9018951F9342
:1045D000CF93DF93CDB7DEB7AA970FB6F894DEBFBF
:1045E0000FBECDBF82E992E02091F100FC01219342
:1045F000CF01F2E08A399F07B9F70E94581E8091D7
:10460000E80083FF1EC180919202909193029A303C
:1046100008F017C1E92FF0E0E85FFA4D0C947D2413
:10462000803899F0823809F00CC1809196028F7021
:10463000873008F006C18093E9008091EB0085FB8C
:10464000882780F91092E90006C080918E0290912F
:104650008F02911182609091E800977F9093E8001B
:104660008093F1001092F1008091E8008E77E5C010
:10467000882309F4D3C0823009F0E3C0809194020A
:104680008111D6C0809196028F702FEF280F2630AF
:1046900008F0D7C08093E9002091EB0020FFC8C04C
:1046A000933031F48091EB0080628093EB00C0C0C6
:1046B0009091EB0090619093EB0021E030E001C01D
:1046C000220F8A95EAF72093EA001092EA0080917F
:1046D000EB008860EACF8111B4C0109194021F777B
:1046E0008091E3008078812B8093E3008091E80043
:1046F000877F8093E8000E9404218091E80080FF7A
:10470000FCCF8091E30080688093E30082E0111188
:1047100083E08093910295C08058823008F091C068
:1047200080919402909195028C3D23E09207A1F52F
:1047300083E08A838AE289834FB7F894DE01139677
:1047400020E03EE051E2E32FF0E050935700E49187
:1047500020FF03C0E295EF703F5FEF708E2F90E077
:10476000EA30C0F0C7968D939D932F5F243159F79F
:104770004FBF8091E800877F8093E8006AE270E095
:10478000CE0101960E9413208091E8008B778093E0
:10479000E80057C0C096E7CF6091960270919702EB
:1047A000AE014F5F5F4F0E944E1FBC01892B09F481
:1047B00048C09091E800977F9093E80089819A81A2
:1047C0000E947120E1CF8038E1F58091E800877F79
:1047D0008093E80080918D028093F10045CF811194
:1047E00030C090919402923060F58091E800877F0C
:1047F0008093E80090938D020E94042180918D02A5
:10480000882311F084E005C08091E30087FDFACF92
:1048100081E0809391020E944E1E13C08091940209
:10482000813079F481E0933009F080E080938F0249
:104830001092E9008091E800877F8093E8000E9451
:1048400004218091E80083FF0AC08091E800877FFF
:104850008093E8008091EB0080628093EB00AA9641
:104860000FB6F894DEBF0FBECDBFDF91CF911F9181
:1048700008950895CF93809191028823A1F0C0916B
:10488000E900CF709091EC00892F817090FD80E855
:10489000C82B1092E9008091E80083FD0E94E72276
:1048A000CF70C093E900CF910895AA1BBB1B51E1C3
:1048B00007C0AA1FBB1FA617B70710F0A61BB70B90
:1048C000881F991F5A95A9F780959095BC01CD0135
:1048D000089597FB072E16F4009407D077FD09D0B2
:1048E0000E94552407FC05D03EF4909581959F4F7A
:1048F0000895709561957F4F0895EE0FFF1F059005
:10490000F491E02D0994FB01DC0102C005900D92A9
:1049100041505040D8F70895F999FECF92BD81BD1E
:10492000F89A992780B50895A6E1B0E044E050E0F8
:104930000C94C624A8E1B0E042E050E00C94C624F8
:10494000262FF999FECF92BD81BDF89A019700B448
:10495000021639F01FBA20BD0FB6F894FA9AF99AE8
:104960000FBE08950396272F0E94A1240E94A02421
:10497000252F0E94A124242F0C94A1240196272FD7
:104980000E94A1240C94A024DC01CB01FC01F99924
:10499000FECF06C0F2BDE1BDF89A319600B40D928B
:1049A00041505040B8F70895F894FFCF4A0A520A90
:1049B000590A5E0A630A680A6D0A720A770A7C0A53
:1049C000810A860A4C0A4C0A4C0A4C0A4C0A4C0AC8
:1049D0004C0A4C0AFA0FFA0F52105210A410C010D1
:1049E00027102710CB10571166116611C21127101E
:1049F0002710CB114E124E1257125712591257123E
:104A0000571257124E124E125E12571257125E1262
:104A1000102338232124382321246B238C232124A1
:044A2000E323EF237A
:104A2400010001000100010001000100010001007A
:104A3400010001000100010000040004041C021430
:104A44000A32110F0514119A1DF91DD81DD41DD059
:104A54001D01E200E900EA00B500B600B700CD0090
:104A64008301CC008A0192019401210223022402D1
:104A74002502260227022A02B300B4006F00700048
:104A8400818283F0F1F4F567F7F6000100FF01007D
:104A9400010000FFFF0000010001FF009196903526
:104AA400E200E900EA00B500B600B700CD008301DA
:104AB400CC008A01920194012102230224022502DE
:104AC400260227022A02B300B4006F00700081821C
:024AD40083005D
:00000001FF
